:020000040000FA
:06000000FE300C303A282E
:08000800A000030EA100831209
:10001000AA1503140B19031000308100A30DA40DC1
:10002000A50DA90B1C282A162508A8002408A7003E
:100030002308A6001930A9008B100B11210E830094
:06004000A00E200E0900D5
:0C007400203084008001840A80300402E7
:10008000031C3C281F30CE000130CA00CB0080305A
:10009000CD000E30F5003230D70083161F308505B5
:1000A000003086050B3087058312850186018701A4
:1000B000103083168E008312703083168F008312E7
:1000C0000030031799000313003003179A0003133D
:1000D0000C30970000309F00003083169F00831281
:1000E000183003179E000313003003179F000313FB
:1000F000803083168100831211309000043092000A
:100100007F308316920083120030950000308316F2
:100110009400831223309400A63083169800831233
:10012000003083169B00831210309800193083161C
:1001300099008312003083168C00831200308316DE
:100140008D00831200308B000D16D22381018E01A9
:100150008F010B118B100B108C018D010D168B175D
:10016000E621A92731175C219D22E920651AF0209C
:10017000E51AEB202A1AF5208F080319B4288F01FD
:10018000E51A0717651A07150025B11B6B21651ABB
:10019000F020E51AEB20AA239B231B227922651A63
:1001A000F020E51AEB204F18A521651AF020E51A7A
:1001B000EB204F18B428AA19E328CC0BB428AA1AAC
:1001C000E7281930A900AA110C30CC00B42854211A
:1001D000B428640008006B080E0203180713080017
:1001E0006B080E020318071108002A12C1302802FA
:1001F000031D0D292708BD002608BC0007303D025D
:100200000319BD27FF303D0203190C29FE303D02C2
:1002100003190C297F23D2234F29280827062602F9
:10022000031D0800F7302802031D19292708BF0005
:100230004F29A1302802031D20292708F0004F294B
:10024000A2302802031D27292708C2004F29A73002
:100250002802031D38292A10A71B2A1427087F39D2
:10026000EA002A1CEA012B142A1C2B10AB154F297B
:10027000C2302802031D4F292708C40064000D1E48
:100280003F298B13440803178D0083168C130C141D
:1002900083120C080313C5008B17CE164F29AA161C
:1002A000AA110A30CC0008004F144F150B12831608
:1002B00005118312051508004F10CF101930A90041
:1002C000AA12AA110A30CC008316051583128B10CE
:1002D0000B110B160800E61C080033080319080070
:1002E00033083602031D7A2934083702031D7A29A0
:1002F000B1130800AF0A01302F02031D8229330811
:100300009300080007302F02031D89293408930049
:1003100008000D302F02031D93293508031908002A
:100320003508930008000E302F02031D0800330823
:10033000B6003408B700B301B401B501AF01B11381
:10034000311F0800B327311308004F19B229C90320
:100350000F304905031D0800C9080319B229051506
:10036000C90E080005114F11CF185C294B1846081B
:10037000CB1847084B1948084D05031DC2294430C6
:10038000C900C5291130C900C5290310CD0C0318B7
:10039000CA2908008030CD000310CB0DCB19D1291C
:1003A00008000130CB001030CE1ACA0041084002CC
:1003B0008030031DCA000310CA0D03184A144A08EE
:1003C0004E050319D129E621CF140800C601C70143
:1003D000C8014A1CF1297730C6004008C700C10097
:1003E000172ACA1CF8296630C6004308C700172A16
:1003F0004A1DFF295530C6007108C700172ACA1DBB
:10040000062A4430C6007608C700172A4A1E0D2A5D
:100410003330C6007808C700172ACA1E08002130EA
:10042000C6004408C7004508C800CE1208004608A8
:100430004706C8000800051CB80A0518B8033808A4
:10044000031940120319B80A3B0838020319401671
:100450000319B803851CB90A8518B90339080319AB
:10046000C0110319B90A3B0839020319C015031951
:10047000B903851DBA0A8519BA033A080319401150
:100480000319BA0A3B083A02031940150319BA03C3
:100490008719C010871DC0143F1886163F1C86128E
:1004A000C219BB23C219582A2A1BBB232A1F0712B1
:1004B000E6195F2ABF1C8613BF188617632ABF1C64
:1004C0008617BF1886133F1F6513401C6A2A3F1BFF
:1004D0006A2AE5177108C01800306619F100C318C0
:1004E000782A2B1C782A053078024310031C431409
:1004F0000800B11B0800E008031D0800310842068F
:10050000013903198A2A301342183017A3273110F2
:10051000421831143108420603390319962A30165D
:10052000A327B110C218B114B2010800301E080090
:10053000B20B08003012A3270800EA080319A72A03
:10054000AB18AF2A6A0895002A18A92A0800950155
:10055000080006162B14AB10421AAB1408002B1D12
:1005600008002B11D518F62AD70BB4283230D70043
:10057000D514AB19CE228B131D3003178D008316B3
:100580008C130C1483120C080313DE006A08950008
:100590002A1C0800AB10421AAB140800AB11213022
:1005A000BF1C013E03178D0083168C130C1483129D
:1005B0000C080313D8008B17203003178D00831607
:1005C0008C130C1483120C080313DC008B175808CF
:1005D0005C07D9005C07DA005C07DB006A087F3C37
:1005E000DD000310DD0C0310DD0C0800DE08031D28
:1005F000FB2ADE03080058087802031C0D2B59085B
:100600007802031C0F2B5A087802031C112B5B087D
:100610007802031C132BD40A152BD00A152BD10AF0
:10062000152BD20A152BD30A152B5008510452044E
:1006300053045404103903190800D601501AD61473
:10064000511A5615521AD615531A5616541AD6164A
:10065000D001D101D201D301D401D5103230D7005D
:100660006A08ED005D075619ED005D07D619ED002B
:100670005D07561AED005D07D61AED006D0895006E
:1006800008000030BD007108BC007F230800F10A9B
:10069000720A71020318F1000800F103720AF11BDB
:1006A000F107080064000D1E532B8B13063003174F
:1006B0008D0083168C130C1483120C0803138B17F4
:1006C0003F1D3030F200F203701B7C2B700871026A
:1006D0000318742B0319742B71087002BF1872026F
:1006E000BF18013EF300080070087102BF1C7202BF
:1006F000BF1C013EF3000800FA30F30008000D12A1
:100700003D08831203178D00831203133C088312E4
:1007100003178C00831603178C130C158B138B1B7C
:100720008E2B55308D00AA308D008C148B170C1138
:10073000831203130800F50BA72B0E30F5009F144E
:100740007603F7009F18A22B2A151E08F6008D309D
:100750009F0008009F149F18AB2B2B158B1383163B
:100760001E0883128B17F8001E08C310031DC31444
:1007700011309F000800AD132D13AD0B0800AC0A1B
:1007800003302C02031C080007121E302E1C0A30F6
:100790002C02031C0800AE0A0130E61AAE00071650
:1007A000AC01080064000D1ED32B8B13003003171F
:1007B0008D0083168C130C1483120C080313F100A4
:1007C0008B138B1BE02B083003178D0083168C13C3
:1007D0000C1483120C080313E6008B171C3003174C
:1007E0008D0083168C130C1483120C080313BB00AA
:1007F0008B1708000708403A870008000708043AEA
:10080000870008000708103A870008000608103A19
:10081000860008000608203A860008000608803A8C
:040820008600080046
:100A0000123060020318E00105308A006008820796
:100A10001A2D2E2DAC2DC42DD02DE92D0E2E222ECB
:100A2000502E8A2EC62EEF2EFF2E172F232F3C2F4F
:100A3000542F592F07170711FB01FC01EB01E51398
:100A40004010C012651B08003F1F080065175223A5
:100A5000F308031908000130E0000800AB1040144F
:100A6000B017A3272A17C31143138B13053003179D
:100A70008D0083168C130C1483120C080313EC00E6
:100A80008B178B13033003178D0083168C130C14F4
:100A900083120C080313F9008B178B130430031710
:100AA0008D0083168C130C1483120C080313FA00A8
:100AB0008B178B130C3003178D0083168C130C14BB
:100AC00083120C080313FD008B178B130D300317D3
:100AD0008D0083168C130C1483120C080313FE0074
:100AE0008B178B130E3003178D0083168C130C1489
:100AF00083120C080313FF008B178B131B30031793
:100B00008D0083168C130C1483120C080313E4005D
:100B10008B170130BF1C013E8B1303178D0083160A
:100B20008C130C1483120C080313EF008B17113075
:100B3000BF1C013E8B1303178D0083168C130C14FE
:100B400083120C080313EE008B176C08E100FF30D2
:100B5000EB000230E0000800E516E10B08006C082D
:100B6000E100EB0B0800E5128B13133003178D0027
:100B700083168C130C1483120C080313E1008B17DB
:100B8000E2010330E000080007130711E20B080040
:100B9000E10B08006C08E100EB010430E000080004
:100BA0006516E10B08006C08E100EB0F0800EB0391
:100BB00065128B13143003178D0083168C130C14DD
:100BC00083120C080313E1008B17E2010530E000EB
:100BD000080007130715E61CF92DE1080319F92D84
:100BE000E61F3016E61B3017A327E20B0800E10BC7
:100BF0000800E61F3012E61B3013A3278B131630B4
:100C000003178D0083168C130C1483120C08031326
:100C1000E1008B17E2010630E0000800E20B08005B
:100C2000E10B08008B13183003178D0083168C130B
:100C30000C1483120C080313E1008B17E201073038
:100C4000E0000800C0160616AB156E08EA00AB14EB
:100C5000661CAB10E51492272B14E20B0800E10B85
:100C600008000130E51BF300AB1001307302031DD7
:100C7000402E6E08EA00AB14661CAB10E51081270D
:100C80008B13193003178D0083168C130C148312E9
:100C90000C080313E1008B17E2010830E0000800A4
:100CA00064277908760203185A2E7F08FC02031C79
:100CB0005F2E08007F08FC070318792E0800FC014E
:100CC0000130E51BF300AB1001307302031D6F2EE2
:100CD0006E08EA00AB14661CAB10E5108127E20B2E
:100CE0000800E10B0800C315F3012A131130E000DE
:100CF0000800FC018B131A3003178D0083168C1328
:100D00000C1483120C080313E1008B17E201093065
:100D1000E000080064277A087602031C942E7F08FE
:100D2000FC02031C992E08007F08FC070318A32E61
:100D30000800FC01E20B0800E10B08004317F30177
:100D40001130E0000800BF1C4723BF184D23F31BE0
:100D5000B62EF30BB62E6E08EA00AB14661CAB1071
:100D6000E51081270A30E000FB0108008B131930E1
:100D700003178D0083168C130C1483120C080313B5
:100D8000E1008B17E2010830E00008002A1D08008E
:100D90002A1176087702031CD22E7D08FB02031C61
:100DA000D72E08007E08FB070318D92E0800FB0188
:100DB0000800FB018712EA012B10AB107B278B1375
:100DC000173003178D0083168C130C1483120C0834
:100DD0000313E1008B17E2010B30E0000800412310
:100DE000C0120612E20B0800B013A327E10B0800A3
:100DF0006C08E100FF30EB000C30E00008006516E5
:100E0000E10B08006C08E100EB0B080065128B1386
:100E1000133003178D0083168C130C1483120C08E7
:100E20000313E1008B17E2010D30E0000800071307
:100E30000711E20B0800E10B08006C08E100EB0170
:100E40000E30E0000800E516E10B08006C08E10038
:100E5000EB0F0800EB03E5128B13153003178D0021
:100E600083168C130C1483120C080313E1008B17E8
:100E7000E2010F30E000080007170711E61C4C2FB5
:100E8000E10803194C2F661F3016661B3017A32785
:100E9000E20B0800E10B0800661F3012661B3013DE
:100EA000A3271030E00008002A137B270030E00061
:100EB00008002A137B27B0138712EA012B10AB100E
:100EC00006120030E0000800E51C0800E40B0800F2
:100ED0008B131B3003178D0083168C130C14831295
:100EE0000C080313E4008B17EA0A6F086A02031D5B
:100EF0000800E51008002430B3000030B400B1173A
:100F000008002430B3008B131E3003178D008316A6
:100F10008C130C1483120C080313B5008B17D727FE
:100F2000B11708002430B3008B131F3003178D0056
:100F300083168C130C1483120C080313B5008B1743
:100F4000D727B11708000630B3003008B400B11736
:100F500008001430AF00FE30B300D930B400FF30C9
:100F6000B500B11708001430AF00FE30B300E53013
:100F7000B400FF30B500B1170800B601FE30B30071
:100F8000A130B400C527B1170800B5013C18B5174A
:100F9000BC1835173C19B516BC1935163C1AB515D1
:100FA000BC1A35153C1BB514BC1B35140800B40124
:100FB0003518B417B51834173519B416B5193416D1
:100FC000351AB415B51A3415351BB414B50108001B
:084000000B00000002000500A6
:02400E00CC03E1
:1042000000007E007E00AA0096000A001800FF0051
:104210008700FF00FF00FF0041002E001400FF0098
:1042200000003200320002001400150016003700B2
:104230000600190080005A00FF0000000100600025
:10424000050040004000FF00FF00FF00FF00FF00EE
:10425000FF00FF00FF00FF00FF00FF00FF00FF0066
:10426000FF00FF00FF00FF00FF00FF00FF00FF0056
:10427000FF00FF00FF00FF00FF00FF00FF00FF0046
:10428000FF00FF00FF00FF00FF00FF00FF00FF0036
:10429000FF00FF00FF00FF00FF00FF00FF00FF0026
:1042A000FF00FF00FF00FF00FF00FF00FF00FF0016
:1042B000FF00FF00FF00FF00FF00FF00FF00FF0006
:1042C000FF00FF00FF00FF00FF00FF00FF00FF00F6
:1042D000FF00FF00FF00FF00FF00FF00FF00FF00E6
:1042E000FF00FF00FF00FF00FF00FF00FF00FF00D6
:1042F000FF00FF00FF00FF00FF00FF00000025009F
:00000001FF
